:020000040000FA
:0600000060283E300130D3
:08000800A000030EA100831209
:1000100005191028831601178312B2308100422877
:100020008316011383120B191C28AE17280A031913
:100030002E17AE192D283B28AE13AE192A282E1FD5
:100040003B28AE1A3B28A701A601A501A801AE01D5
:10005000AE164228F030AE0542282D152E13AE12F2
:100060002708AB002608AA002508A9002808AC002C
:10007000F030AE0542282E0DA80DA50DA60DA70D3A
:10008000AE1AAE0A8B100B11210E8300A00E200EAB
:02009000090065
:1000C000203084008001840A80300402031C6228EE
:1000D000BD2283160C3085058701831285018701B7
:1000E0000730990000309A00103083168E0083127A
:1000F000603083168F0083120030831691009F00BA
:100100008312C83083168100831231309000003092
:1001100083168C00831210308B00BD1B9128851D27
:1001200042233D1BBE013D1BBF013D1F2B2381010F
:100130008E018F010B118B100B108C018B17B020CF
:100140002D19B2208F22B30BAD280310851903148B
:10015000BA0DF0303A020319E621BD186A239F2830
:100160006400080029083F3C0319BE282B082A0612
:1001700029062C02031D2D11031D08002D1101302D
:10018000B7008B132030370783169B001C141A0806
:100190008312A4001030370783169B001C141A0822
:1001A0008312A3000030370783169B001C141A0823
:1001B0008312A2008B1724082B02031DE0292308B9
:1001C0002A02031DE029013009303702031D1629D8
:1001D00029083F3C0319002940302906E039031D56
:1001E000F6283F1FF6283F13AD1704296030290673
:1001F000E039031D04293F1B04293F17AD170429CB
:10020000AC1F3F13AC1B3F1780302906F039031D8C
:100210000D29BF1F0D29BF13AD1790302906F039E6
:10022000031D1629BF1B1629BF17AD17A91FE029EB
:10023000291BE02922082906F039A91EE039031DEF
:10024000E029220829050F390319802901303702D6
:10025000031D2F293E182F293E14AD17D32202303B
:100260003702031D3829BE183829BE14AD17D52210
:1002700003303702031D41293E1941293E15AD17B0
:10028000D72204303702031D4A29BE194A29BE1558
:10029000AD17D92205303702031D53293E1A5329C1
:1002A0003E16AD17DB2206303702031D5C29BE1A4D
:1002B0005C29BE16AD17DD2207303702031D652904
:1002C0003E1B65293E17AD17DF2208303702031D9C
:1002D0006E29BE1B6E29BE17AD17E1220930370209
:1002E000031D77293F1877293F14AD17E3220A3001
:1002F0003702031D8029BF188029BF14AD17E722DC
:10030000290922050F390319E02901303702031D9D
:100310008E293E1C8E293E10AD17EB22023037028B
:10032000031D9729BE1C9729BE10AD17ED2203307F
:100330003702031DA0293E1DA0293E11AD17EF2253
:1003400004303702031DA929BE1DA929BE11AD170E
:10035000F12205303702031DB2293E1EB2293E129A
:10036000AD17F32206303702031DBB29BE1EBB2981
:10037000BE12AD17F52207303702031DC4293E1FF8
:10038000C4293E13AD17F72208303702031DCD29CB
:10039000BE1FCD29BE13AD17F92209303702031D48
:1003A000D6293F1CD6293F10AD17FB220A30370251
:1003B000031DDF29BF1CDF29BF10AD17FF22E02975
:1003C000B70A0B30370203180800C128B601B30181
:1003D0009630B4000130B5000130B70085018701C7
:1003E000AD136F22B020B30B302A0310851903140C
:1003F000BA0DF0303A0203195F2AB40B302A0130EB
:10040000370203190323023037020319072303308D
:10041000370203190B230430370203190F23053069
:100420003702031913230630370203191723073045
:10043000370203191B230830370203191F23093021
:100440003702031923230A303702031927233708F9
:10045000B6080319B60003192E2AB6039630B40065
:100460002D1DF2292D11A91FF229291BF229A91EE0
:1004700029120F3029050319F229B9012918B90ADF
:10048000A918B90A2919B90AA919B90AB918F22972
:100490003919F2298B1320303707BC002B08BB0019
:1004A0009D2210303707BC002A08BB009D22003077
:1004B0003707BC002908BB009D228B1769228501E4
:1004C0008701B70AB6010B303702031CF2292B2330
:1004D00008000A303702031908008501870114302B
:1004E000B90033300F1E85000F1A8501FF300F1A37
:1004F00087000F1E8701B0202D1D712A2D11290A9A
:100500000319862AA91F712A291B712A0F30290570
:10051000031D6F2AB90B712A850187010800AD1FE1
:100520000800AD131030BC003E08BB009D223030E7
:10053000BC003F08BB009D2208003C088B138316BB
:100540009B001C141A0883128B173B020319080026
:100550008B133B0883161C159A0083123C088316E4
:100560009B0055309D00AA309D009C1464009C188F
:10057000B62A1C1183128B170800831600309B00CB
:100580001C141A088312BD00831610309B001C1423
:100590001A088312BE00831630309B001C141A0800
:1005A0008312BF0008000516080085160800051410
:1005B00008008514080087140800071508000714B0
:1005C000080087160800BD18080007160800BD18A7
:1005D000080087150800051208008512080005109C
:1005E0000800851008008710080007110800071090
:1005F000080087120800BD18080007120800BD187F
:100600000800871108000508103A85000800050851
:10061000203A850008000508013A85000800050811
:10062000023A850008000708023A87000800070818
:10063000043A870008000708013A87000800070805
:10064000203A870008000708103A870008000708CA
:10065000083A870008003E180516BE1885163E1990
:100660000514BE1985143E1A8714BE1A07153E1BC1
:100670000714BE1B8716BD1808003F180716BF18C1
:1006800087150800B601B301B4013D1C4A2B3D108B
:10069000BD144D2BC030BD053D143D083F39B6009B
:1006A0006400522B532B542B552B562B3330B41B39
:1006B0008500B41F8501B30B502BB40B502B0310D6
:1006C000B60CB608031D502B0030BC003D08BB0023
:1006D0009D220800BF1F752B3F1B07123F1B87156C
:1006E0003F1F07163F1F87110800071287110800D8
:084000000200000006000200AE
:02400E00CC33B1
:1042000001008100820084008800B100B200B40087
:10421000B800A100A200FF00FF00FF00FF00FF00A8
:104220000000010001000100010001000100010087
:10423000010001000100FF00FF00FF00FF00FF0080
:10424000010000000000000000000000000000006D
:10425000000000000000FF00FF00FF00FF00FF0063
:104260000000FF00FF00FF00FF00FF00FF00FF0055
:10427000FF00FF00FF00FF00FF00FF00FF00FF0046
:10428000FF00FF00FF00FF00FF00FF00FF00FF0036
:10429000FF00FF00FF00FF00FF00FF00FF00FF0026
:1042A000FF00FF00FF00FF00FF00FF00FF00FF0016
:1042B000FF00FF00FF00FF00FF00FF00FF00FF0006
:1042C000FF00FF00FF00FF00FF00FF00FF00FF00F6
:1042D000FF00FF00FF00FF00FF00FF00FF00FF00E6
:1042E000FF00FF00FF00FF00FF00FF00FF00FF00D6
:1042F000FF00FF00FF00FF00FF00FF00FF00DD00E8
:00000001FF
